:030000000219FDE5
:03000B000200AA46
:03002B0002019936
:03005B0002034F4E
:0300730002033550
:1000800002030406080C10182030406080040608A3
:100090000C10182030406080A0C000070F1F3F0DDB
:1000A0000D0403060D0503030202C2AF306308C24C
:1000B00063857C8AD2AF32C0D0C0E0206227E525BC
:1000C0006002E473E525F4C3334009758A00D26306
:1000D000F57C01D6F58A758B00758D00D262D0E073
:1000E000D0D0D2AF32C3E526334009758A00D2633F
:1000F000F57C01F6F58AC262E526F4603B306803C0
:10010000207213758B00758D00D0E0D0D0C292C2E2
:1001100094C296D2AF32C292C294C296206E0C2084
:100120006609740AD5E0FDE57E4290758B00758DF9
:1001300000D0E0D0D0D2AF32758A00D263757C0097
:10014000C28DD262212B01C4306805206602D29292
:1001500001C4306805206602D29401C430680520CD
:100160006602D29601C4C29330680A2066077408FA
:10017000D5E0FDD29201C4C29530680A20660774AA
:1001800008D5E0FDD29401C4C29730680A20660702
:100190007408D5E0FDD29601C4C2AFC2AD53E6EFFC
:1001A000C0D0C0E0D2D3D2AFE57D6009E57A60056A
:1001B000757A00413E757A01C2CEE52A6007207447
:1001C00049152A410A7800790020742EE580307E96
:1001D00001F430E60278FF53DACF207E0343DA20C1
:1001E000307E0343DA10C2D8C271E580307E01F45C
:1001F00030E60279FFC3E89970CB306103752A407D
:10020000207403752A40885FD27020740DE52B603E
:1002100004152B411A43DA01C2D8207002412DA8DF
:100220005F206102C270207402412B88227882B65E
:100230000403852224C3E52594404002D26420CFE4
:100240000AD0E0D0D043E610D2AD32C2CF053AE5B5
:100250007D6009E57B6005757B00612B757B01780E
:1002600002E52A6005307402152AC3E55F94014057
:10027000057562004187756300756C00E5622401B5
:10028000F56250037562FF7982B7020D306D1DC3B0
:10029000E52294324016854D227982B7030E306DE7
:1002A0000BC3E52294324004798E8722C3E523955F
:1002B0002260084004152341BB0523D8CA056CE51C
:1002C0006C7002156CD56D63756D017805C3E56CB6
:1002D000956E4057C3E56C956F50087801756D03B6
:1002E0000202EFC3E56C957050057801756D01C38E
:1002F000E5659524401E7982B704026120206D14C3
:10030000852465E56C046003856E6C756D0175234D
:100310003C02032BE5652850057565FF6120F565F6
:10032000E5650470067563FF756CFFD0E0D0D043BF
:10033000E610D2AD32C2AFC0D053E67FC260759135
:1003400000855694855795759104D0D0D2AF32C2AE
:10035000AF53E6EFC2ADC0D0C0E0C0F0D2D3D2AF51
:10036000A8FBA9FCE57D6007C3E913F9E813F8C20F
:10037000D830710261C153DACF207E0343DA1030E6
:100380007E0343DA20D271E580307E01F420E6025C
:10039000619888278928A1A653DACF207E0343DA03
:1003A00020307E0343DA10C2D8C271307402A192A9
:1003B0007800E580307E01F430E602A192885FA1EA
:1003C0007A53DACF207E0343DA20307E0343DA10FB
:1003D000C271206102819A53DACF207E0343DA1082
:1003E000307E0343DA20C2D8D271885A895BC3E8D1
:1003F0009558F8E99559F97B007E087A00C3E8948E
:100400008CE994005005755E00818C882178A2E605
:10041000A8216055C3E894C8E994005008E4D2E4E8
:10042000FB7A0A8167C3E89468E994015008E4D232
:10043000E3FB7A0F8167C3E894D0E994025008E4A3
:10044000D2E2FB7A1E8167C3E894A0E994055008C4
:10045000E4D2E1FB7A3C8167C3E89498E9940850C0
:1004600008E4D2E0FB7A787E00C3E8955CFCE9956D
:0F0470005DFD30E70AECF42401FCEDF43400FDEF
:10047F00755E00C3EC9AED9E5003755E01885C8932
:10048F005D855A58855B597802A17AC3E89527F89C
:10049F00E99528F9307C02A15E307B02A15E307AAB
:1004AF0002A15720750281BDE9FDE8FC81DCE9C39B
:1004BF0013F9E813F8307902A157E9C313F9E813D8
:1004CF00F8307802A157E9C313FDE813FC20612C23
:1004DF00C3EC941CED9402400281F3ED701EC3EC4B
:1004EF0094C850180529E52970021529C3E52994E8
:1004FF000A5002A192755F00D270A192E5296002A5
:10050F0015297400207F037896E624FAFEE4340060
:10051F00FFC3EC9EFCED9FFD500678007900A15EB5
:10052F00C3EC94FFED9400400678FF7900A15EECD8
:10053F008575F0A4C5F0A2F733F8790040030205E2
:10054F007A78FF790002057AE9C313F9E813F830D6
:10055F007C0EE9600278FFC3E81338F8E43400F941
:10056F00C3E894FFE99400400278FF885FD27020BF
:10057F006102A192741FF4552F4BF52FC274EB70CB
:10058F0002D274752A40307403752A0A306102A1B1
:10059F00A620740353DAFE207403752B20D0F0D0FD
:1005AF00E0D0D0D2AD43E6103279010205D67903FF
:1005BF000205D6790A0205D6791E0205D67964029C
:1005CF0005D679C80205D67817E4D5E0FDD8FAD953
:1005DF00F6227A147B780205FD7A107B8C0205FDDA
:1005EF007A0D7BB40205FD7A0B7BC80205FD7902FB
:1005FF00B27DE4C295D5E0FDD294D5E0FDC294D58D
:10060F00E0FDD295D5E0FDD292E576D5E0FDC29220
:10061F007496D5E0FDD9D9EAF8D5E0FDD8FBDBCE4D
:10062F00C29522C37C007D0075F00005F0EA33FA15
:10063F00EB33FB50F6EB13FBEA13FAC3E9FFE8FECB
:10064F00E89AF8E99BF95004EFF9EEF8B3EC33FCB4
:10065F00ED33FDD5F0DFEDF9ECF822E889F08A20D3
:10066F00D2D4F8A9F07B0030F70B7BFFF42401F80C
:10067F00E9F43400F9E88520F0A4ADF0F8E985201D
:10068F00F0A4AFF0FEED2EF974003FFA7C04C3EA3C
:10069F0013FAE913F9E813F8DCF48BF030F70AE8F2
:1006AF00F42401F8E9F43400F9E889F0C2D4F8A988
:1006BF00F0227882B60403020760C3E55F94194005
:1006CF001EE52D54067018206D3678057994E714C1
:1006DF006007780A1460027812C3E54198401F3012
:1006EF006D09856765756CFF756D01852224E4F5CD
:1006FF0045F546F547F548F549C26D020760D26DDD
:10070F007994E7147013E523F43333F913F8E954AC
:10071F000104F9E854FE020754E714147014E5239A
:10072F00F4333333F913F8E9540304F9E854FC02B2
:10073F00075CE523F433333333F913F8E954070433
:10074F0004F9E854F8C39440F8E99400F98845890E
:10075F004622C3E54113F9E54013F8C3E54598F880
:10076F00E54699F9500CC3E89480E994FF401602CE
:10077F000798C3E8947FE994005003020798787FA5
:10078F007900020798788079FF884A894B22E54AD9
:10079F002547F8E54B3548F9854B20E4300701F440
:1007AF003549FA30E709C3EA94F040150207D6C37A
:1007BF00EA940F50030207D678FF79FF7A0F0207EA
:1007CF00D6780079007AF0C3E5249564500AC37493
:1007DF00019524500B0207F4E54B20E70E0207F4B6
:1007EF00E54B30E706884789488A492278A4E6FA1C
:1007FF00C3E54A33F8E54B33F912066AE930E70BE4
:10080F00C3E89480E994FF4013012FC3E8947FE974
:10081F0094005002012F787F7900012F788079FFA3
:10082F00E820E715C3E52398F84009C3E894014091
:10083F00030208567801020856E8F424012523F82C
:10084F00400302085678FF884C2278A5E6FAA8489C
:10085F00A94912066AE930E70CC3E89401E994FF4D
:0E086F00401602088BC3E894FFE99400500382
:10087D0002088B78FF790002088B780179FFE92057
:10088D00E715C3E54C98F84009C3E894014003020D
:10089D0008B278010208B2E8F42401254CF84003AF
:1008AD000208B278FF88242278FFC26420693D20B7
:1008BD006A12D264C3E541940A4009C3E525944008
:1008CD005002C26479A1E76023E541601F74FF8582
:1008DD0041F0848539F0306A0375F005A4F8C5F050
:1008ED00600278FFC3E895675002A867886622C347
:1008FD00E54094C8E5419400E566500314210D04CC
:10090D006002F566227883E6F520120FD275E89025
:10091D001205B875E890E5E820ECFBA8BDA9BE125C
:10092D001070757155757200C3740013FD745560A8
:10093D006613FC74552CFC74003DFDECFAEDFBC305
:10094D00E89AE99B4014E5712455F571E572340080
:10095D00F572EA2CFAEB3DFB80E5AE71AF72C3E5A3
:10096D007213F9E57113F8C3E913F9E813F87A0373
:10097D00C3E913F9E813F8DAF7AA201A70097571AB
:10098D00007572000209A41AEA6008EE28FEEF391C
:10099D00FFDAF88E718F722275E890227883E6FF68
:1009AD00E5E820ECF7A8BDA9BE0573C3E57394086F
:1009BD004052757300E9FA79A0E76044EA7007E5E3
:1009CD0074601B0209DFC3E895746010E57450066E
:1009DD00600C140209EB0460F90209EBE574F5747F
:1009ED00C39472401B7564C0C39404401375648036
:1009FD00C39404400B756440C394044003756400B4
:100A0D0075BB0922EFC39401601F7455601BC3E8C9
:100A1D0094FFE994035012C3E89571E9957250095A
:100A2D00E564600C1564020A3DE564F4600205643A
:100A3D00A864C3E524985002A824C3E89565400A2C
:100A4D00A865E565F4600385656488258826E573EA
:100A5D00B4070375BB1022743279A687F0A4C5F0D4
:100A6D00A2F733F8C3E895644002A864882288246D
:100A7D00882588268867227540007541F022C2AF0F
:100A8D0075C820A8CCA9CDAA3A30CF010A75C824C3
:100A9D00D2AFC3EA13FAE913F9E813F8AB3BAC3C58
:100AAD00883B893CC3E89BF8E99C20690A547FF98F
:100ABD0030670261AE610BAD3D8A3DF9EA9D547F11
:100ACD00FA600478FF79FFAE3EAF3F8B3E8C3FC39B
:100ADD00EC9FFCC3E99CF542A83BA93CC3E89EF8FA
:100AED00E99FF9C3E54113FBE54013FAE82AF54008
:100AFD00E93BF54150067540FF7541FF6155AA4030
:100B0D00AB41AC40AD417E047F02C3EB9404400287
:100B1D001E1FC3EB940840021E1FC3ED13FDEC1303
:100B2D00FCDEF7C3EA9CFAEB9DFBEF6009C3E9130A
:100B3D00F9E813F8DFF7EA28FAEB39FB8A408B4125
:100B4D0050067BFF8B408B41C3EB94025002D26762
:100B5D003069047F0361807892E6FFC3E5379482A4
:100B6D0040110FC3E53794A040010FC3EF94064029
:100B7D00027F057E02E541C4540FF9E541C454F0EE
:100B8D00F8E540C4540F28F8C3E89EFAE99400FB39
:100B9D004009C3EA9402EB940050047A02E4FB612D
:100BAD00FAAA40AB41EBC4FEEAC4540F4EFCC3EAB3
:100BBD009CFAEB9400FBC3E813C313F8EA28FAEB95
:100BCD003400FB8A408B41C3EB94024002C267782C
:100BDD0002EBC4FE7B00EAC4540F4EFAC3EA98FA46
:100BED004005C3940250027A027892E6FF3060020B
:100BFD0061FA855256855357D26043E680C3E49A15
:100C0D00F8E49BF9C3E833F8E933F9306702819BC7
:100C1D00E8FAE9FBD3E913FDE813FC88528953C3C5
:100C2D00EF94036038EF20E00DE82CF8E93DF9EC86
:100C3D00FAEDFB020C56E828F8E939F9C3E824026D
:100C4D00F8E93400F97AFE7BFFC3EF9403400E8A76
:100C5D00548B55884E894F8C508D5181CF88548936
:0F0C6D00558A4E8B4F8C508D51306920C3E53323
:100C7C0094034019E542A2E713F8E555F424013832
:100C8C00400B20E7087554FFF42401F55581CFE89B
:100C9C00FAD3E813FC8852C3EF94036020EF20E0F2
:100CAC0007E82CF8ECFA81BBE8282402F87AFEC39A
:100CBC00EF940340088A54884E8C5081CF88548A14
:100CCC004E8C50E56BC3335002646BF56B30600295
:100CDC0081D9753404D26043E680E52D5406601F3B
:100CEC00A840A941C2AF53E67F759100C3E498F5C3
:100CFC0094E499F595759104D26043E680D2AF22C5
:100D0C00D265754400752000306B03752040020DD0
:100D1C002BD265754400752040306B03752000D2D2
:100D2C00AF7801206722E52D54066002C265C3E549
:100D3C0041940540137802940540087803940540CB
:100D4C00027806306902780A206019E54460153093
:100D5C00690AC3E53394034003D53406D2AFD26C91
:100D6C00C10D91E1D2AF0000C2AF20672AE541C3AB
:100D7C00FB940F40027B0FEB240530730123306A88
:100D8C0002742820620123F93069027982E58D13FF
:100D9C00E58B13C39940B10544E59B5440B5200243
:100DAC00A1F730690A08C3E8940A400108A154204D
:100DBC006502A12BC26553E67F75910030671075F3
:100DCC0094007595FC759104D26043E680A12BAE1E
:100DDC0040AF41C3EE33FEEF33FF50047EFF7FFF85
:100DEC00C3E49EF594E49FF595A1D1C3E533940239
:100DFC005002A12B306502A12BD802C10BA154C209
:100E0C006C53E67F759100855494855595759104C6
:100E1C00854E56854F57D26043E680D2AFE52D54B0
:100E2C00066008206A020533020E47306C0D206BF9
:100E3C000A206507158115810216D02278003064CE
:100E4C00053065027801E53775F007A4F9E5F0285F
:100E5C00F5F0E9A2F013A2F113A2F213F537C39443
:100E6C00785003753778C3E53795384008D266C299
:100E7C0092C294C296306002C181855056855157FA
:100E8C00D26043E68022D287207D11C2AF75430227
:100E9C00C295D293D2AF759F8002106DC2AF7543CD
:100EAC0002C295D297D2AF759F8002106DC2873067
:100EBC007243207D20C2AF754303900177757E206D
:100ECC00C296C297306204D294C1D9D295D2AF7572
:100EDC009F8902106DC2AF754303900177757E2018
:100EEC00C292C293306204D294C1F9D295D2AF753A
:100EFC009F8102106D207D17C2AF75430390015284
:100F0C00C296306202D294D2AF759F8902106DC224
:100F1C00AF754303900152C292306202D294D2AFA9
:100F2C00759F8102106DD287207D11C2AF7543046D
:100F3C00C293D297D2AF759F8102106DC2AF754329
:100F4C0004C297D293D2AF759F8902106DC28730BD
:100F5C007243207D20C2AF754305900166757E08F3
:100F6C00C294C295306204D292E179D293D2AF7519
:100F7C009F8002106DC2AF754305900188757E800D
:100F8C00C294C295306204D296E199D297D2AF75D1
:100F9C009F8002106D207D17C2AF754305900148EC
:100FAC00C294306202D292D2AF759F8002106DC291
:100FBC00AF75430590015CC2943062EBD296D2AF10
:100FCC00759F8002106DD287207D11C2AF754306CC
:100FDC00C297D295D2AF759F8902106DC2AF75437F
:100FEC0006C293D295D2AF759F8102106DC2873025
:100FFC007242207D20C2AF754301900188757E80BE
:10100C00C292C293306204D2960119D297D2AF75B4
:10101C009F8102106DC2AF754301900166757E0809
:10102C00C296C297306204D2920139D293D2AF7574
:10103C009F89016D207D16C2AF75430190015CC282
:10104C0092306202D296D2AF759F81016DC2AF759C
:10105C004301900148C296306202D292D2AF759F82
:0E106C0089C26622900146757E00C292C2942F
:10107A00C296C293C295C297C26222788076070846
:10108A0076070876010876040876FF0876FF087660
:10109A0009087602087601087601788C76010876C6
:1010AA00000876B40876FF0876FF0876FF0876030C
:1010BA000876FF0876010876FF0876250876D008B4
:1010CA0076780876C80876040876FF0876010876E6
:1010DA000008767A08760A0876010876010876000A
:1010EA000876FF227887E6FFC272BF0302D27278BF
:1010FA0088C27DE630E102D27DC27E7889E630E19F
:10110A0002D27EC3EF94026008758E01D273021177
:10111A0020758E00C273227880E61490008093783E
:10112A00A4F67881E6149000809378A5F67886E68E
:10113A001490008D9378A6F6789FE6F8700108C39C
:10114A00E8941140027811E82828F56E256E256E7C
:10115A0028F56F256E2828F570789CE67538FF7596
:10116A00390CB402067538A075390AB40306753805
:10117A008275390578A3E61490009A93F56911707F
:10118A0022C2A4C2A0789DE6B40104D2A4C2A0B42B
:10119A000204C2A4D2A0227896E6FA7897E6FB78EF
:1011AA0088E6B40305C3EB940EFB307F047A007B18
:1011BA00FFC3EB9AFCC3948250027C8275750005CA
:1011CA0075EC8575F0A4C3E5F0947D40F222D27FD8
:1011DA0031A11205C77A007B007C101205BDE55FBC
:1011EA002AFA74003BFBDCF37C04C3EB13FBEA131F
:1011FA00FADCF7FEC27F31A122E5EF20E603752073
:10120A00000520903FFFE520146006901FFF146040
:10121A00009304600375EF1253D9BF7581C043FF71
:10122A00801205B875EF0243B203E5B3240420E740
:10123A000DF521E5E320E0068521B343E3011170B2
:10124A007580FF75A48075F1F075D4BF759002752D
:10125A00A5FC75F2FD75D50275A61175A0EE75F39C
:10126A00F175E241E4F8F6D8FD756B0111851217A4
:10127A001F78988676753001C2AF1205D11205E142
:10128A001205C71205E81205C71205EF1205C712A3
:10129A0018411205D11205D11205CCC2AF78FA79DC
:1012AA00FA308607D9FBD8F7021C0011EE3121313A
:1012BA008B31A178988676117075A90075B68075FC
:1012CA007D0075885075891275C82475910475D882
:1012DA004075A82275B80275E690759B80759D00C9
:1012EA0075D10E75BCC075BB0975BA1175E8801247
:1012FA0005B8D2AF12091253DACF207E0343DA209F
:10130A00307E0343DA1043DA01C2D8C2711205D122
:10131A00D2617B037A0CE55E70077A0CDB0302125A
:10132A00A51205C72070030212A5C270E55FC39417
:10133A000240E1E52F541F856160F561B560D5DA99
:10134A00D5C26153DACF207E0343DA20307E0343CD
:10135A00DA10C2D8C27178A2E67008D274E52F54A6
:10136A00E0F52FC2757529001205CC307409C3E562
:10137A0029940A4002D2751205BD780230740278A7
:10138A0000C3E55F9840F0C2AF1205E11205E11211
:10139A0005E1D2AF1205D1754D001205BD788CE674
:1013AA00C39401500302147AE530C3940150030236
:1013BA00147A207435C3E55F94FF500302147AC28D
:1013CA00AF1205F6D2AF1205CCC3E55F940150EF18
:1013DA00C2AF1205E11205C21205E1D2AF1205CC65
:1013EA00C3E55F94FF40E90218C67F05D27F31A1A9
:1013FA001205CCC2AFC27F31A1AE5FC3E55F947F55
:10140A00D2AF40761205B8C2AF1205F6D2AFDFDC12
:10141A0031D8C3EE94057897F61205D112176012E7
:10142A0018497F0AD27F31A11205CCC2AFC27F31DF
:10143A00A1AE5FC3E55F947FD2AF50E61205B8C292
:10144A00AF1205E11205C21205E1D2AFDFD631D8DB
:10145A00EE24057896F61205D11217601218781242
:0D146A0005CC31A1C3E55F94FF500261BCC9
:101477000218C6C3E55F954D4003855F4D1205CC45
:1014870078017988E7B403027805C3E55F984002DD
:1014970061A4C2AF1205F61205F61205F6D2AF1215
:1014A70005D1753000E4F531F5320531E531F470D9
:1014B700390532789AE67819146012783214600D7B
:1014C700787D14600878FA146003753200C3E5323A
:1014D70098401715327531B478998676C2AF1205E0
:1014E700F6D2AF789886761205CC1205C2E52A7037
:1014F7000530740241A578012074027806C3E55FC0
:101507009840A71205CCE52A70030212A5C2AF11B5
:1015170070E4F522F523F524F525F526F56AD2AF13
:101527007885E6C333F568E4F545F546F547F548AC
:10153700F549F573F52CF52DF53775730875BB105F
:101547001205B81209A5E5E820ECFBA8BDA9BEE97C
:101557007001F888741209A975730875BB1078872C
:10156700E6FE760211EE7887EEF6C2AF7564FF12DB
:101577000A64852264852265852266D2AF752201B9
:1015870075240175250175260185636C756D0175D7
:10159700B69075A903757D017888E6B40307C27D07
:1015A700307602D27DD268D269753300120FD2121B
:1015B7000FF9120A84120A8B120A84120A8B120A72
:1015C700840215D7C2AF11EED2AF75730075BB0990
:1015D700120D1D1206C1120E48120E92120A8B121C
:1015E7000D0C306D031207612067031208B53067D1
:1015F700031208FC120E48120EB9120A8B120D1DA7
:10160700306D0312079D120E48120F32120A8B1209
:101617000D0C306D031207FB120E48120F59120AF8
:101627008B120D1D306D03120859120E48120FD27E
:10163700120A8B1209A5120D0C120E48120FF9127D
:1016470009A9120A8B30692F206B2C85676485677F
:101657006585636C756D0179187A0CC3E53399401C
:1016670009C269D26A8A3502167EC3E55F940140D2
:10167700030215D70216D8306A1B206B18E53514FC
:101687007004C26AA1CBF535C3E55F94014003023C
:1016970015D70216D8753600C3E56294014009854F
:1016A700676585636C756D01C3E56278FA985021AB
:1016B700307404E52A601A78F0306B058567647822
:1016C70020C3E541985002A1D70536E55F6002C106
:1016D700DB753600C2AF11707887E6FE760211EE31
:1016E7007887EEF6E4F522F523F524F525F526F5BA
:1016F70068C26875A90075B680757D00D2AF1205FE
:10170700B81170307406E52A700241A5788DE6C3DA
:1017170094014002618181AC901A0D78201217A2C2
:10172700E520B4A50CA31217A2E520B45A030217AB
:1017370040118512176002175F901A0378807B0AA1
:101747001217A2A308DBF9901A0F788C7B181217CF
:10175700A2A308DBF9901A2722C2AF1217E11217CA
:10176700BB901A00740E1217A7A374041217A7A32D
:1017770074141217A7901A0378807B0A1217A6A36E
:1017870008DBF9901A0F788C7B181217A6A308DBD1
:10179700F91217F41217D2901A2722E493F622E6C9
:1017A700438F01538FFD75EF0275B7A575B7F1F03C
:1017B700538FFE22438F02438F0175EF0275B7A542
:1017C70075B7F1901A0DF0538FFC22901A0D74A57E
:1017D700F1A7901A0E745AF1A7227A3079D078209F
:1017E700901A40F1A2E520F709A3DAF7227A3079B7
:1017F700D0901A40E7F1A709A3DAF922AB77A878C6
:10180700BB01027980BB02027981BB03027982BBEB
:1018170004027994BB05027983BB06027986BB076C
:10182700027992BB08027987BB0902799CBB0A023D
:101837007988BB0B027989E8F7227C051205D1DC90
:10184700FB22C2AF1205E11205E81205EF1205F6F9
:101857001205C21205E11205E81205EF1205F6128C
:0E18670005C21205E11205E81205EF1205F6A2
:10187500D2AF22C2AF1205F61205EF1205E8120526
:10188500E11205C21205F61205EF1205E81205E18F
:101895001205C21205F61205EF1205E81205E1D28E
:1018A500AF22AE77AF78C2AF1205E11205E112059E
:1018B500E11205C2DEF21205F61205C2DFF8D2AF5B
:1018C500221149114111417577017578017579002A
:1018D50011A77C05AD5F1205D1C3ED955F70F5C30A
:1018E500E55F9401400AC3E55F94FF4033021903A5
:1018F50011031217601149C2AF75EF121141DCD403
:101905000579C3E5799403500280C511410578E551
:10191500771490009F93F808C3E57898500280AD3E
:10192500114111410577C3E577940C5002809B1254
:0C1935001085121760C2AF75EF1211414F
:0319FD00021203D0
:101A00000E041407070104FFFF09020101A55A0192
:101A100000B4FFFFFF03FF01FF25D078C804FF01DA
:081A200000FF0A010100FFFFB5
:101A400023506C6174696E756D3530417633232097
:101A500023424C48454C492346333930232020202B
:101A60002020202020202020202020202020202076
:101C0000C2AFC2D353D9BF7581C043B20343FF8073
:101C1000752438752503B1C975EF0275E24043F1AB
:101C20004053A4BF75D400D2867DFA780379E67C50
:101C300010752200752300901DD67B0675249875BB
:101C400025013086028142208608D8FBD9F9DCF7CD
:101C500081B4308608D8FBD9F9DCF781B4B189E4C6
:101C600093A3C39A6004DDC381B4DBDBB17B600264
:101C7000812B7B08E493FAA3B15CDBF87A30B15C8A
:101C8000752200752300B17BEAFCEBFDC3ED94FEE9
:101C9000400EB17B8A278B28ED30E0048A828B834B
:101CA000B17B7AC270D8C3ED94FE601350CEBD00F4
:101CB00025EC60097520007521FF0200008100A855
:101CC00027A9280809D804D90281D3B17FEA89AAB3
:101CD000F281C50D81A0C3ED94035049EDA2E092BD
:101CE000007AC5C3E5829400E583941C50902000DF
:101CF00010438F02438F0175B7A575B7F1F030001F
:101D00001FA827A9280809438F01538FFDD804D99C
:101D100002A12089AAE275B7A575B7F1F0A3A10DBC
:101D2000538FFC817C7AC1BD030CE493A3FAB140CC
:101D3000DCF8B138817C817EAA22AB23B15CEBFA5E
:101D4000EA6222752608C3E52313F523E52213F57D
:101D50002250066323A0632201D526EAB1C9B1C986
:101D600075260AEAF4200102D286300102C286B149
:101D7000C9C3134002C201D526EB22B17FEAFB2082
:101D80008602A17F308602A184752608AE24AF2585
:101D9000C3EF13FFEE13FEB1CDB1C9C3EA13308612
:101DA000024480FA30E703632201C3E52313F523DD
:101DB000E52213F52250066323A0632201D526D91C
:101DC000E52265236523F52222AE24AF250E0FDE22
:101DD000FEDFFCD20122424C48656C693437316326
:041DE000F390060175
:00000001FF
